

Microchip MPLAB XC8 Assembler V2.32 build 20210201212658 
                                                                                               Thu Jan 13 12:02:14 2022

Microchip MPLAB XC8 C Compiler v2.32 (Free license) build 20210201212658 Og1 
     1                           	processor	18F4580
     2                           	fnconf	rparam,??,?,0
     3                           	pagewidth 120
     4                           	opt	flic
     5                           	psect	cinit,global,reloc=2,class=CODE,delta=1
     6                           	psect	cstackCOMRAM,global,class=COMRAM,space=1,delta=1,lowdata,noexec
     7                           	psect	text0,global,reloc=2,class=CODE,delta=1
     8                           	psect	text1,global,reloc=2,class=CODE,delta=1
     9                           	psect	intsave_regs,global,class=BIGRAM,space=1,delta=1,noexec
    10                           	psect	rparam,global,class=COMRAM,space=1,delta=1,noexec
    11                           	psect	idloc,global,abs,ovrld,class=IDLOC,space=5,delta=1,noexec
    12                           	psect	config,global,abs,ovrld,class=CONFIG,space=4,delta=1,noexec
    13  0000                     
    14                           ; Version 2.20
    15                           ; Generated 12/02/2020 GMT
    16                           ; 
    17                           ; Copyright © 2020, Microchip Technology Inc. and its subsidiaries ("Microchip")
    18                           ; All rights reserved.
    19                           ; 
    20                           ; This software is developed by Microchip Technology Inc. and its subsidiaries ("Microch
      +                          ip").
    21                           ; 
    22                           ; Redistribution and use in source and binary forms, with or without modification, are
    23                           ; permitted provided that the following conditions are met:
    24                           ; 
    25                           ;     1. Redistributions of source code must retain the above copyright notice, this lis
      +                          t of
    26                           ;        conditions and the following disclaimer.
    27                           ; 
    28                           ;     2. Redistributions in binary form must reproduce the above copyright notice, this 
      +                          list
    29                           ;        of conditions and the following disclaimer in the documentation and/or other
    30                           ;        materials provided with the distribution.
    31                           ; 
    32                           ;     3. Microchip's name may not be used to endorse or promote products derived from th
      +                          is
    33                           ;        software without specific prior written permission.
    34                           ; 
    35                           ; THIS SOFTWARE IS PROVIDED BY MICROCHIP "AS IS" AND ANY EXPRESS OR IMPLIED WARRANTIES,
    36                           ; INCLUDING, BUT NOT LIMITED TO, THE IMPLIED WARRANTIES OF MERCHANTABILITY AND FITNESS F
      +                          OR
    37                           ; PURPOSE ARE DISCLAIMED.  IN NO EVENT SHALL MICROCHIP BE LIABLE FOR ANY DIRECT, INDIREC
      +                          T,
    38                           ; INCIDENTAL, SPECIAL, EXEMPLARY, OR CONSEQUENTIAL DAMAGES (INCLUDING BUT NOT LIMITED TO
    39                           ; PROCUREMENT OF SUBSTITUTE GOODS OR SERVICES; LOSS OF USE, DATA OR PROFITS; OR BUSINESS
    40                           ; INTERRUPTION) HOWSOEVER CAUSED AND ON ANY THEORY OF LIABILITY, WHETHER IN CONTRACT, ST
      +                          RICT
    41                           ; LIABILITY, OR TORT (INCLUDING NEGLIGENCE OR OTHERWISE) ARISING IN ANY WAY OUT OF THE U
      +                          SE OF
    42                           ; THIS SOFTWARE, EVEN IF ADVISED OF THE POSSIBILITY OF SUCH DAMAGE.
    43                           ; 
    44                           ; 
    45                           ; Code-generator required, PIC18F4580 Definitions
    46                           ; 
    47                           ; SFR Addresses
    48  0000                     _PR2	set	4043
    49  0000                     _T2CON	set	4042
    50  0000                     _PORTA	set	3968
    51  0000                     _TRISA	set	3986
    52  0000                     _TMR2IF	set	31985
    53  0000                     _RA0	set	31744
    54                           
    55                           ; #config settings
    56                           
    57                           	psect	cinit
    58  007FC4                     __pcinit:
    59                           	callstack 0
    60  007FC4                     start_initialization:
    61                           	callstack 0
    62  007FC4                     __initialization:
    63                           	callstack 0
    64  007FC4                     end_of_initialization:
    65                           	callstack 0
    66  007FC4                     __end_of__initialization:
    67                           	callstack 0
    68  007FC4  0100               	movlb	0
    69  007FC6  EFEE  F03F         	goto	_main	;jump to C main() function
    70                           
    71                           	psect	cstackCOMRAM
    72  000000                     __pcstackCOMRAM:
    73                           	callstack 0
    74  000000                     
    75                           ; 1 bytes @ 0x0
    76 ;;
    77 ;;Main: autosize = 0, tempsize = 0, incstack = 0, save=0
    78 ;;
    79 ;; *************** function _main *****************
    80 ;; Defined at:
    81 ;;		line 4 in file "TImer.c"
    82 ;; Parameters:    Size  Location     Type
    83 ;;		None
    84 ;; Auto vars:     Size  Location     Type
    85 ;;		None
    86 ;; Return value:  Size  Location     Type
    87 ;;                  1    wreg      void 
    88 ;; Registers used:
    89 ;;		wreg, status,2, cstack
    90 ;; Tracked objects:
    91 ;;		On entry : 0/0
    92 ;;		On exit  : 0/0
    93 ;;		Unchanged: 0/0
    94 ;; Data sizes:     COMRAM   BANK0   BANK1   BANK2   BANK3   BANK4   BANK5
    95 ;;      Params:         0       0       0       0       0       0       0
    96 ;;      Locals:         0       0       0       0       0       0       0
    97 ;;      Temps:          0       0       0       0       0       0       0
    98 ;;      Totals:         0       0       0       0       0       0       0
    99 ;;Total ram usage:        0 bytes
   100 ;; Hardware stack levels required when called: 1
   101 ;; This function calls:
   102 ;;		_timer
   103 ;; This function is called by:
   104 ;;		Startup code after reset
   105 ;; This function uses a non-reentrant model
   106 ;;
   107                           
   108                           	psect	text0
   109  007FDC                     __ptext0:
   110                           	callstack 0
   111  007FDC                     _main:
   112                           	callstack 30
   113  007FDC                     
   114                           ;TImer.c: 5:     TRISA=0x00;
   115  007FDC  0E00               	movlw	0
   116  007FDE  6E92               	movwf	146,c	;volatile
   117                           
   118                           ;TImer.c: 6:     PORTA=0x00;
   119  007FE0  0E00               	movlw	0
   120  007FE2  6E80               	movwf	128,c	;volatile
   121                           
   122                           ;TImer.c: 7:     T2CON=0x7E;
   123  007FE4  0E7E               	movlw	126
   124  007FE6  6ECA               	movwf	202,c	;volatile
   125                           
   126                           ;TImer.c: 8:     PR2=195;
   127  007FE8  0EC3               	movlw	195
   128  007FEA  6ECB               	movwf	203,c	;volatile
   129  007FEC                     l708:
   130                           
   131                           ;TImer.c: 10:         RA0=1;
   132  007FEC  8080               	bsf	3968,0,c	;volatile
   133  007FEE                     
   134                           ;TImer.c: 11:         timer();
   135  007FEE  ECE5  F03F         	call	_timer	;wreg free
   136  007FF2                     
   137                           ;TImer.c: 12:         RA0=0;
   138  007FF2  9080               	bcf	3968,0,c	;volatile
   139  007FF4                     
   140                           ;TImer.c: 13:         timer();
   141  007FF4  ECE5  F03F         	call	_timer	;wreg free
   142  007FF8  EFF6  F03F         	goto	l708
   143  007FFC  EF00  F000         	goto	start
   144  008000                     __end_of_main:
   145                           	callstack 0
   146                           
   147 ;; *************** function _timer *****************
   148 ;; Defined at:
   149 ;;		line 16 in file "TImer.c"
   150 ;; Parameters:    Size  Location     Type
   151 ;;		None
   152 ;; Auto vars:     Size  Location     Type
   153 ;;		None
   154 ;; Return value:  Size  Location     Type
   155 ;;                  1    wreg      void 
   156 ;; Registers used:
   157 ;;		None
   158 ;; Tracked objects:
   159 ;;		On entry : 0/0
   160 ;;		On exit  : 0/0
   161 ;;		Unchanged: 0/0
   162 ;; Data sizes:     COMRAM   BANK0   BANK1   BANK2   BANK3   BANK4   BANK5
   163 ;;      Params:         0       0       0       0       0       0       0
   164 ;;      Locals:         0       0       0       0       0       0       0
   165 ;;      Temps:          0       0       0       0       0       0       0
   166 ;;      Totals:         0       0       0       0       0       0       0
   167 ;;Total ram usage:        0 bytes
   168 ;; Hardware stack levels used: 1
   169 ;; This function calls:
   170 ;;		Nothing
   171 ;; This function is called by:
   172 ;;		_main
   173 ;; This function uses a non-reentrant model
   174 ;;
   175                           
   176                           	psect	text1
   177  007FCA                     __ptext1:
   178                           	callstack 0
   179  007FCA                     _timer:
   180                           	callstack 30
   181  007FCA                     l25:
   182  007FCA  A29E               	btfss	3998,1,c	;volatile
   183  007FCC  EFEA  F03F         	goto	u11
   184  007FD0  EFEC  F03F         	goto	u10
   185  007FD4                     u11:
   186  007FD4  EFE5  F03F         	goto	l25
   187  007FD8                     u10:
   188  007FD8                     
   189                           ;TImer.c: 19:         TMR2IF=0;
   190  007FD8  929E               	bcf	3998,1,c	;volatile
   191  007FDA  0012               	return		;funcret
   192  007FDC                     __end_of_timer:
   193                           	callstack 0
   194  0000                     
   195                           	psect	rparam
   196  0000                     
   197                           	psect	idloc
   198                           
   199                           ;Config register IDLOC0 @ 0x200000
   200                           ;	unspecified, using default values
   201  200000                     	org	2097152
   202  200000  FF                 	db	255
   203                           
   204                           ;Config register IDLOC1 @ 0x200001
   205                           ;	unspecified, using default values
   206  200001                     	org	2097153
   207  200001  FF                 	db	255
   208                           
   209                           ;Config register IDLOC2 @ 0x200002
   210                           ;	unspecified, using default values
   211  200002                     	org	2097154
   212  200002  FF                 	db	255
   213                           
   214                           ;Config register IDLOC3 @ 0x200003
   215                           ;	unspecified, using default values
   216  200003                     	org	2097155
   217  200003  FF                 	db	255
   218                           
   219                           ;Config register IDLOC4 @ 0x200004
   220                           ;	unspecified, using default values
   221  200004                     	org	2097156
   222  200004  FF                 	db	255
   223                           
   224                           ;Config register IDLOC5 @ 0x200005
   225                           ;	unspecified, using default values
   226  200005                     	org	2097157
   227  200005  FF                 	db	255
   228                           
   229                           ;Config register IDLOC6 @ 0x200006
   230                           ;	unspecified, using default values
   231  200006                     	org	2097158
   232  200006  FF                 	db	255
   233                           
   234                           ;Config register IDLOC7 @ 0x200007
   235                           ;	unspecified, using default values
   236  200007                     	org	2097159
   237  200007  FF                 	db	255
   238                           
   239                           	psect	config
   240                           
   241                           ; Padding undefined space
   242  300000                     	org	3145728
   243  300000  FF                 	db	255
   244                           
   245                           ;Config register CONFIG1H @ 0x300001
   246                           ;	unspecified, using default values
   247                           ;	Oscillator Selection bits
   248                           ;	OSC = 0x7, unprogrammed default
   249                           ;	Fail-Safe Clock Monitor Enable bit
   250                           ;	FCMEN = 0x0, unprogrammed default
   251                           ;	Internal/External Oscillator Switchover bit
   252                           ;	IESO = 0x0, unprogrammed default
   253  300001                     	org	3145729
   254  300001  07                 	db	7
   255                           
   256                           ;Config register CONFIG2L @ 0x300002
   257                           ;	unspecified, using default values
   258                           ;	Power-up Timer Enable bit
   259                           ;	PWRT = 0x1, unprogrammed default
   260                           ;	Brown-out Reset Enable bits
   261                           ;	BOREN = 0x3, unprogrammed default
   262                           ;	Brown-out Reset Voltage bits
   263                           ;	BORV = 0x3, unprogrammed default
   264  300002                     	org	3145730
   265  300002  1F                 	db	31
   266                           
   267                           ;Config register CONFIG2H @ 0x300003
   268                           ;	unspecified, using default values
   269                           ;	Watchdog Timer Enable bit
   270                           ;	WDT = 0x1, unprogrammed default
   271                           ;	Watchdog Timer Postscale Select bits
   272                           ;	WDTPS = 0xF, unprogrammed default
   273  300003                     	org	3145731
   274  300003  1F                 	db	31
   275                           
   276                           ; Padding undefined space
   277  300004                     	org	3145732
   278  300004  FF                 	db	255
   279                           
   280                           ;Config register CONFIG3H @ 0x300005
   281                           ;	unspecified, using default values
   282                           ;	PORTB A/D Enable bit
   283                           ;	PBADEN = 0x1, unprogrammed default
   284                           ;	Low-Power Timer 1 Oscillator Enable bit
   285                           ;	LPT1OSC = 0x0, unprogrammed default
   286                           ;	MCLR Pin Enable bit
   287                           ;	MCLRE = 0x1, unprogrammed default
   288  300005                     	org	3145733
   289  300005  82                 	db	130
   290                           
   291                           ;Config register CONFIG4L @ 0x300006
   292                           ;	unspecified, using default values
   293                           ;	Stack Full/Underflow Reset Enable bit
   294                           ;	STVREN = 0x1, unprogrammed default
   295                           ;	Single-Supply ICSP Enable bit
   296                           ;	LVP = 0x1, unprogrammed default
   297                           ;	Boot Block Size Select bit
   298                           ;	BBSIZ = 0x0, unprogrammed default
   299                           ;	Extended Instruction Set Enable bit
   300                           ;	XINST = 0x0, unprogrammed default
   301                           ;	Background Debugger Enable bit
   302                           ;	DEBUG = 0x1, unprogrammed default
   303  300006                     	org	3145734
   304  300006  85                 	db	133
   305                           
   306                           ; Padding undefined space
   307  300007                     	org	3145735
   308  300007  FF                 	db	255
   309                           
   310                           ;Config register CONFIG5L @ 0x300008
   311                           ;	unspecified, using default values
   312                           ;	Code Protection bit
   313                           ;	CP0 = 0x1, unprogrammed default
   314                           ;	Code Protection bit
   315                           ;	CP1 = 0x1, unprogrammed default
   316                           ;	Code Protection bit
   317                           ;	CP2 = 0x1, unprogrammed default
   318                           ;	Code Protection bit
   319                           ;	CP3 = 0x1, unprogrammed default
   320  300008                     	org	3145736
   321  300008  0F                 	db	15
   322                           
   323                           ;Config register CONFIG5H @ 0x300009
   324                           ;	unspecified, using default values
   325                           ;	Boot Block Code Protection bit
   326                           ;	CPB = 0x1, unprogrammed default
   327                           ;	Data EEPROM Code Protection bit
   328                           ;	CPD = 0x1, unprogrammed default
   329  300009                     	org	3145737
   330  300009  C0                 	db	192
   331                           
   332                           ;Config register CONFIG6L @ 0x30000A
   333                           ;	unspecified, using default values
   334                           ;	Write Protection bit
   335                           ;	WRT0 = 0x1, unprogrammed default
   336                           ;	Write Protection bit
   337                           ;	WRT1 = 0x1, unprogrammed default
   338                           ;	Write Protection bit
   339                           ;	WRT2 = 0x1, unprogrammed default
   340                           ;	Write Protection bit
   341                           ;	WRT3 = 0x1, unprogrammed default
   342  30000A                     	org	3145738
   343  30000A  0F                 	db	15
   344                           
   345                           ;Config register CONFIG6H @ 0x30000B
   346                           ;	unspecified, using default values
   347                           ;	Configuration Register Write Protection bit
   348                           ;	WRTC = 0x1, unprogrammed default
   349                           ;	Boot Block Write Protection bit
   350                           ;	WRTB = 0x1, unprogrammed default
   351                           ;	Data EEPROM Write Protection bit
   352                           ;	WRTD = 0x1, unprogrammed default
   353  30000B                     	org	3145739
   354  30000B  E0                 	db	224
   355                           
   356                           ;Config register CONFIG7L @ 0x30000C
   357                           ;	unspecified, using default values
   358                           ;	Table Read Protection bit
   359                           ;	EBTR0 = 0x1, unprogrammed default
   360                           ;	Table Read Protection bit
   361                           ;	EBTR1 = 0x1, unprogrammed default
   362                           ;	Table Read Protection bit
   363                           ;	EBTR2 = 0x1, unprogrammed default
   364                           ;	Table Read Protection bit
   365                           ;	EBTR3 = 0x1, unprogrammed default
   366  30000C                     	org	3145740
   367  30000C  0F                 	db	15
   368                           
   369                           ;Config register CONFIG7H @ 0x30000D
   370                           ;	unspecified, using default values
   371                           ;	Boot Block Table Read Protection bit
   372                           ;	EBTRB = 0x1, unprogrammed default
   373  30000D                     	org	3145741
   374  30000D  40                 	db	64
   375                           tosu	equ	0xFFF
   376                           tosh	equ	0xFFE
   377                           tosl	equ	0xFFD
   378                           stkptr	equ	0xFFC
   379                           pclatu	equ	0xFFB
   380                           pclath	equ	0xFFA
   381                           pcl	equ	0xFF9
   382                           tblptru	equ	0xFF8
   383                           tblptrh	equ	0xFF7
   384                           tblptrl	equ	0xFF6
   385                           tablat	equ	0xFF5
   386                           prodh	equ	0xFF4
   387                           prodl	equ	0xFF3
   388                           indf0	equ	0xFEF
   389                           postinc0	equ	0xFEE
   390                           postdec0	equ	0xFED
   391                           preinc0	equ	0xFEC
   392                           plusw0	equ	0xFEB
   393                           fsr0h	equ	0xFEA
   394                           fsr0l	equ	0xFE9
   395                           wreg	equ	0xFE8
   396                           indf1	equ	0xFE7
   397                           postinc1	equ	0xFE6
   398                           postdec1	equ	0xFE5
   399                           preinc1	equ	0xFE4
   400                           plusw1	equ	0xFE3
   401                           fsr1h	equ	0xFE2
   402                           fsr1l	equ	0xFE1
   403                           bsr	equ	0xFE0
   404                           indf2	equ	0xFDF
   405                           postinc2	equ	0xFDE
   406                           postdec2	equ	0xFDD
   407                           preinc2	equ	0xFDC
   408                           plusw2	equ	0xFDB
   409                           fsr2h	equ	0xFDA
   410                           fsr2l	equ	0xFD9
   411                           status	equ	0xFD8

Data Sizes:
    Strings     0
    Constant    0
    Data        0
    BSS         0
    Persistent  0
    Stack       0

Auto Spaces:
    Space          Size  Autos    Used
    COMRAM           95      0       0
    BANK0           160      0       0
    BANK1           256      0       0
    BANK2           256      0       0
    BANK3           256      0       0
    BANK4           256      0       0
    BANK5           256      0       0

Pointer List with Targets:

    None.

Critical Paths under _main in COMRAM

    None.

Critical Paths under _main in BANK0

    None.

Critical Paths under _main in BANK1

    None.

Critical Paths under _main in BANK2

    None.

Critical Paths under _main in BANK3

    None.

Critical Paths under _main in BANK4

    None.

Critical Paths under _main in BANK5

    None.

Call Graph Tables:

 ---------------------------------------------------------------------------------
 (Depth) Function   	        Calls       Base Space   Used Autos Params    Refs
 ---------------------------------------------------------------------------------
 (0) _main                                                 0     0      0       0
                              _timer
 ---------------------------------------------------------------------------------
 (1) _timer                                                0     0      0       0
 ---------------------------------------------------------------------------------
 Estimated maximum stack depth 1
 ---------------------------------------------------------------------------------

 Call Graph Graphs:

 _main (ROOT)
   _timer

 Address spaces:
Name               Size   Autos  Total    Cost      Usage
BITCOMRAM           5F      0       0       0        0.0%
EEDATA             100      0       0       0        0.0%
NULL                 0      0       0       0        0.0%
CODE                 0      0       0       0        0.0%
COMRAM              5F      0       0       1        0.0%
STACK                0      0       0       2        0.0%
ABS                  0      0       0       3        0.0%
BITBANK0            A0      0       0       4        0.0%
BANK0               A0      0       0       5        0.0%
BITBANK1           100      0       0       6        0.0%
BANK1              100      0       0       7        0.0%
BITBANK2           100      0       0       8        0.0%
BANK2              100      0       0       9        0.0%
BITBANK3           100      0       0      10        0.0%
BANK3              100      0       0      11        0.0%
BITBANK4           100      0       0      12        0.0%
BANK4              100      0       0      13        0.0%
BITBANK5           100      0       0      14        0.0%
BANK5              100      0       0      15        0.0%
BIGRAM             5FF      0       0      16        0.0%
DATA                 0      0       0      17        0.0%
BITSFR_3             0      0       0     200        0.0%
SFR_3                0      0       0     200        0.0%
BITSFR_2             0      0       0     200        0.0%
SFR_2                0      0       0     200        0.0%
BITSFR_1             0      0       0     200        0.0%
SFR_1                0      0       0     200        0.0%
BITSFR               0      0       0     200        0.0%
SFR                  0      0       0     200        0.0%


Microchip Technology PIC18 Macro Assembler V2.32 build 20210201212658 
Symbol Table                                                                                   Thu Jan 13 12:02:14 2022

                     l25 7FCA                       l27 7FD8                       l28 7FDA  
                     u10 7FD8                       u11 7FD4                      l710 7FEE  
                    l704 7FCA                      l712 7FF2                      l714 7FF4  
                    l706 7FDC                      l708 7FEC                      _RA0 007C00  
                    _PR2 000FCB                     _main 7FDC                     start 0000  
           ___param_bank 000000                    ?_main 0000                    _T2CON 000FCA  
                  _PORTA 000F80                    _TRISA 000F92                    _timer 7FCA  
        __initialization 7FC4             __end_of_main 8000                   ??_main 0000  
          __activetblptr 000000                   ?_timer 0000                   _TMR2IF 007CF1  
                 isa$std 000001               __accesstop 0060  __end_of__initialization 7FC4  
          ___rparam_used 000001           __pcstackCOMRAM 0000            __end_of_timer 7FDC  
                ??_timer 0000                  __Hparam 0000                  __Lparam 0000  
                __pcinit 7FC4                  __ramtop 0600                  __ptext0 7FDC  
                __ptext1 7FCA     end_of_initialization 7FC4      start_initialization 7FC4  
         __size_of_timer 0012                 __Hrparam 0000                 __Lrparam 0000  
          __size_of_main 0024                 isa$xinst 000000  
